:100000000C94A3000C94CB000C94CB000C94CB006C
:100010000C94CB000C94CB000C94CB000C94CB0034
:100020000C94CB000C94CB000C94CB000C94CB0024
:100030000C94CB000C94CB000C94CB000C94CB0014
:100040000C941F060C94CB000C94CB000C94CB00AA
:100050000C94CB000C94CB000C94CB000C94CB00F4
:100060000C94CB000C94CB0007634236B79BD8A707
:100070001A39685618AEBAAB558C1D3CB7CC5763CD
:10008000BD6DEDFD753EF6177231BF000000803F7B
:1000900008000000BE922449123EABAAAA2ABECD97
:1000A000CCCC4C3E00000080BEABAAAAAA3E000009
:1000B0000000BF000000803F000000000008417801
:1000C000D3BB4387D1133D190E3CC3BD4282AD2B38
:1000D0003E68EC8276BED98FE1A93E4C80EFFFBE30
:1000E00001C4FF7F3F00000000000000000023006B
:1000F0002600290000000000240027002A0000003C
:100100000000250028002B00040404040404040457
:1001100002020202020203030303030301020408B2
:100120001020408001020408102001020408102061
:1001300000000008000201000003040700000000A6
:1001400000000000420A11241FBECFEFD8E0DEBF3E
:10015000CDBF11E0A0E0B1E0E0E5FEE102C0059016
:100160000D92A031B107D9F727E0A0E1B1E001C0BD
:100170001D92A136B207E1F710E0C3EAD0E004C057
:100180002197FE010E94200FC23AD107C9F70E94B1
:1001900069060C94260F0C940000833081F028F43B
:1001A000813099F08230A9F008958730A9F0883025
:1001B000C9F08430B1F4809180008F7D03C08091BC
:1001C00080008F7780938000089584B58F7784BDF9
:1001D000089584B58F7DFBCF8091B0008F77809399
:1001E000B00008958091B0008F7DF9CF1F93CF9319
:1001F000DF93E3E3F1E09491EFE1F1E0D491EBE000
:10020000F1E0C491CC23B9F0182F992319F0892F6C
:100210000E94CD00EC2FF0E0EE0FFF1FE250FF4FE9
:10022000A591B4918FB7F894EC91111108C0D095B5
:10023000DE23DC938FBFDF91CF911F910895DE2BDA
:10024000F8CFCF93DF9390E0FC01E45EFE4F249162
:10025000885F9E4FFC0184918823C9F090E0880F4D
:10026000991FFC01EC50FF4FA591B491FC01E250A5
:10027000FF4FC591D49161110DC09FB7F8948C9137
:10028000209582238C938881282328839FBFDF9128
:10029000CF910895623051F49FB7F8943C91822F2A
:1002A000809583238C93E8812E2BEFCF8FB7F89422
:1002B000EC912E2B2C938FBFEACF8E5080648093CD
:1002C0007C0080917A00806480937A0080917A002B
:1002D00086FDFCCF809178009091790008953FB71A
:1002E000F89480915D0790915E07A0915F07B091AF
:1002F000600726B5A89B05C02F3F19F00196A11DE8
:10030000B11D3FBFBA2FA92F982F8827BC01CD015F
:10031000620F711D811D911D42E0660F771F881FBE
:10032000991F4A95D1F708952FB7F894609159070E
:1003300070915A0780915B0790915C072FBF0895D9
:100340002F923F924F925F926F927F928F929F92E5
:10035000AF92BF92CF92DF92EF92FF92CF93DF9353
:1003600000D000D0CDB7DEB73C014A015B01CB0124
:10037000BA010E94410C6B019B012F5F3F4F2F3F41
:10038000310519F014F030E020E0F601EE0FFF1F08
:10039000E60DF71D20803180512C412C220F331F98
:1003A000260D371DF9016081718190E080E06219AE
:1003B0007309840995090E94790C69837A838B8378
:1003C0009C83B601DD0C880B990B0E94790C9B0174
:1003D000AC01C501B4010E945D0B9B01AC016981B8
:1003E0007A818B819C810E942E0D0E94410CDC0140
:1003F000CB01820D931DA41DB51D0097F1E0AF0741
:10040000B10524F08FEF9FEFA0E0B0E0B7FF03C08D
:1004100080E090E0DC010F900F900F900F90DF9143
:10042000CF91FF90EF90DF90CF90BF90AF909F90D3
:100430008F907F906F905F904F903F902F90089596
:100440002F923F924F925F926F927F928F929F92E4
:10045000AF92BF92CF92DF92EF92FF920F931F93D2
:10046000CF93DF93CDB7DEB7C25DD1090FB6F89455
:10047000DEBF0FBECDBFCD53DF4F8883C35CD040FE
:10048000C953DF4F9883C75CD0408B015E0121E6E2
:10049000A20EB11CD12CC12C7501F8EE4F2EF3E049
:1004A0005F2E612C712CC016D106C4F40E94A20AE2
:1004B000A30192010E94FA0A0E94790C20E030E028
:1004C0004AE754E40E94CF0BD5016D937D938D9341
:1004D0009D935D01BFEFCB1ADB0AE5CF4801012EEA
:1004E000000CAA08BB0860E070E0CB0110161106F2
:1004F00034F40E94A20AA50194010E94FA0A660F30
:10050000771F660F771F6E0D7F1DFB011082118212
:100510001282138260E070E0CB011016110634F4F1
:100520000E94A20AA50194010E94FA0A660F771F91
:10053000660F771F6E0D7F1D80E090E0A0E8BFE39F
:10054000FB0180839183A283B3839E012F5F3F4F82
:100550006901CF53DF4F39832883C15CD040312CF0
:10056000212C412C512C320156E9852E912CA12CA5
:10057000B12C2016310674F50E94A20AA50194013F
:100580000E94FA0A6E5C7F4F8F4F9F4F0E94790C3A
:1005900020E030E04AE754E40E94CF0B9B01AC011D
:1005A000C301B2010E945E0B2B013C01CF53DF4F10
:1005B000A881B981C15CD0404D925D926D927D92CF
:1005C000CF53DF4FB983A883C15CD040BFEF2B1A54
:1005D0003B0ACFCFB12CA12CA016B106C4F4F60172
:1005E00061917191819191916F014F01F4E08F1AA6
:1005F0009108A30192010E94CF0BD4016D937D93CA
:100600008D939C931397BFEFAB1ABB0AE5CF0150B4
:100610001109F7014081518162817381C801880FFE
:10062000991F880F991FE80FF91F40835183628338
:100630007383E1E0F0E0EC0FFD1FE80FF91F80E0AD
:1006400090E0A0E8BFE380839183A283B38360E05E
:1006500070E0CB01101611064CF40E94A20A98011A
:10066000012E000C440B550B0E94FA0AC353DF4FB6
:1006700079836883CD5CD0400E94A20A20EA30E0F2
:1006800040E050E00E94FA0A605571098109910921
:100690000E94790C20E030E048EC52E40E94CF0B3D
:1006A000C153DF4F688379838A839B83CF5CD040BB
:1006B000CD53DF4FF881C35CD040C553DF4FF88383
:1006C000CB5CD040C953DF4F2881C75CD040C453B6
:1006D000DF4F2883CC5CD040CF53DF4F1982188284
:1006E000C15CD040CF53DF4FA881B981C15CD040FD
:1006F000BD01BB0F880B990B0E94790C20E030E004
:100700004FE753E40E94CF0B2B013C016E01B5E093
:10071000CB0ED11C312C212C7101EFEFEE1AFE0A09
:10072000201631066CF4D6012D913D914D915D91CD
:100730006D01C301B2010E94290D18160CF43DC1D0
:100740006801E016F1060CF467017101EE0CFF1C64
:10075000EE0CFF1CE1E0F0E0EC0FFD1FEE0DFF1DC5
:1007600080809180A280B380A5019401C301B20171
:100770000E945D0B2B013C01CC0CDD1CCC0CDD1C64
:10078000E1E0F0E0EC0FFD1FEC0DFD1DA501940173
:1007900060817181828193810E945D0B9B01AC011C
:1007A000C301B2010E94CF0B4B015C01E1E6F0E016
:1007B000EC0FFD1FEE0DFF1D80819181A281B381A1
:1007C000CD53DF4F88839983AA83BB83C35CD0401A
:1007D000A501940160E070E080E89FE30E945D0B5A
:1007E0002B013C01A1E6B0E0AC0FBD1FCA0EDB1E21
:1007F000D6018D919D910D90BC91A02DC953DF4FD5
:1008000088839983AA83BB83C75CD040C353DF4FDF
:10081000E881F981CD5CD040E215F30509F0D3C041
:100820009C01AD01CD53DF4F688179818A819B8125
:10083000C35CD0400E945E0B20E030E040E05FE30C
:100840000E942E0DC153DF4F288139814A815B817F
:10085000CF5CD0400E945E0B6B017C0120E030E059
:10086000A9010E94CA0B87FDAAC020E030E040E841
:100870005FE3C701B6010E94290D181634F4C12C9C
:10088000D12C80E8E82E8FE3F82EA3019201C3015A
:10089000B2010E945E0BA50194010E942E0DA701DA
:1008A00096010E942E0D6B017C01A3019201C301F0
:1008B000B2010E942E0DCD53DF4F288139814A812C
:1008C0005B81C35CD0400E942E0D9B01AC01C7012F
:1008D000B6010E945E0B6B017C01A5019401C5016C
:1008E000B4010E942E0DC953DF4F288139814A81FE
:1008F0005B81C75CD0400E942E0D9B01AC01C701FB
:10090000B6010E945E0B6B017C0120E030E0A90182
:100910000E94CA0B70E060E087FD16C020E030E066
:1009200040E85FE3C701B6010E94290D6FEF7FEF3A
:10093000181654F020E03FEF4FE757E4C701B60127
:100940000E942E0D0E94480CC553DF4FA881B9812B
:10095000CB5CD0406D937D93C553DF4FB983A883A3
:10096000CB5CD040CF53DF4FE881F981C15CD040F0
:100970003196CF53DF4FF983E883C15CD040E11556
:10098000F14009F0AFCECE52DF4F0FB6F894DEBF84
:100990000FBECDBFDF91CF911F910F91FF90EF90D0
:1009A000DF90CF90BF90AF909F908F907F906F908F
:1009B0005F904F903F902F9008951701ADCEC12CBE
:1009C000D12C760162CFCD53DF4F288139814A8106
:1009D0005B81C35CD040C301B2010E942E0D6B014C
:1009E0007C01C953DF4F288139814A815B81C75C13
:1009F000D040C501B4017FCFCF92DF92EF92FF923A
:100A00000F931F93CF93DF938C01EB0188818111AA
:100A10006CC00E94A20A20E137E240E050E00E9450
:100A2000FA0A0E94790C6B017C01D801ED91FC91CE
:100A300020E030E040EA50E460817181828193815E
:100A40000E942E0D9B01AC01C701B6010E94CA0B8A
:100A500087FF48C081E088830E94A20A28E230E034
:100A600040E050E00E94FA0A665F7F4F8F4F9F4F31
:100A70000E94790C20E030E048EC52E40E94CF0B59
:100A800069837A838B839C830E94A20A20EF3AE0D9
:100A900040E050E00E94FA0A68517C4F8F4F9F4F10
:100AA0000E94790C6B017C01D8011296ED91FC91AA
:100AB0002DEC3CEC4CEC5DE3608171818281938193
:100AC0000E945E0B9B01AC01C701B6010E94CF0BD7
:100AD0006D837E838F8398870E94940169877A87CC
:100AE0008B879C8788818823A9F00E9494010985BF
:100AF0001A852B853C85601B710B820B930B0E9422
:100B0000770C2D813E814F8158850E94290D181642
:100B10000CF41882DF91CF911F910F91FF90EF900D
:100B2000DF90CF900895CF92DF92EF92FF9281E015
:100B30000E94F60081E080934B070E94940160932D
:100B40004707709348078093490790934A0780E1CD
:100B50000E945D019C01990F440B550B211584E007
:100B600038074105510524F02FEF33E040E050E015
:100B700057FF03C020E030E0A901A9E0B0E00E94E7
:100B8000190B2FEF33E040E050E00E94FA0A6901B0
:100B90007A0183E0C80ED11CE11CF11C85E10E94A2
:100BA0005D01BC01990F880B990B611571058105D9
:100BB000910511F00E94F10AB60180E195E00E94D2
:100BC000200284E10E945D01BC01990F880B990B02
:100BD000611571058105910511F00E94F10AB601B8
:100BE00080E193E00E9420020E946F01611571056F
:100BF0008105910511F00E94F10AB60180E191E0B2
:100C00000E942002109210071092110710921207F2
:100C100010921307109214071092150710921607DE
:100C200010921707109218071092190710921A07BE
:100C300010921B07FF90EF90DF90CF9008951F92C6
:100C40000F920FB60F9211242F933F938F939F9380
:100C5000AF93BF938091590790915A07A0915B077A
:100C6000B0915C073091580723E0230F2D3758F5DA
:100C70000196A11DB11D20935807809359079093A9
:100C80005A07A0935B07B0935C0780915D07909132
:100C90005E07A0915F07B09160070196A11DB11D8D
:100CA00080935D0790935E07A0935F07B093600702
:100CB000BF91AF919F918F913F912F910F900FBE58
:100CC0000F901F90189526E8230F0296A11DB11DC5
:100CD000D2CFCF93DF93CDB7DEB760970FB6F8943E
:100CE000DEBF0FBECDBF789484B5826084BD84B56D
:100CF000816084BD85B5826085BD85B5816085BD17
:100D000080916E00816080936E00109281008091CE
:100D10008100826080938100809181008160809356
:100D2000810000E810E08091800081608093800065
:100D30008091B10084608093B1008091B0008160A7
:100D40008093B00080917A00846080937A008091D3
:100D50007A00826080937A0080917A00816080932B
:100D60007A0080917A00806880937A001092C100A6
:100D700060E08EE00E94210160E08FE00E9421018E
:100D800060E080E10E94210160E081E10E94210198
:100D900062E084E00E94210161E083E00E94210181
:100DA00061E089E00E94210161E08AE00E94210166
:100DB00061E08BE00E94210181EA8093800089E05C
:100DC0008093810083E88093B00082E08093B1003B
:100DD000109389000093880010938B0000938A0081
:100DE00080E88093B30085E10E945D01BC01990F0A
:100DF000880B990B611571058105910511F00E9411
:100E0000F10A0E9493051E0129E0220E311C00E028
:100E100010E00E9494014B015C01E4E3F1E0849155
:100E2000E0E2F1E0E490ECE0F1E0F490FF2079F012
:100E300081110E94CD00EF2DF0E0EE0FFF1FE65173
:100E4000FF4FA591B4918C91E82281E009F480E0F4
:100E5000109256071092570790915507891751F035
:100E6000809355078092500790925107A0925207A5
:100E7000B09253078091500790915107A09152076B
:100E8000B0915307881A990AAA0ABB0A80914C07A5
:100E900090914D07A0914E07B0914F078815990585
:100EA000AA05BB05B0F49091540780915507981797
:100EB00081F080935407911103C021E0813009F043
:100EC00020E020935607913009F4811190E090932F
:100ED00057078091570781110E94930580914B0716
:100EE0008823C1F00E949401C0904707D090480722
:100EF000E0904907F0904A076C197D098E099F0917
:100F0000693C71058105910528F080E00E94F6009A
:100F100010924B078EE00E945D01BC01990F880B77
:100F2000990B0E94790C20E030EC4FE754E40E94CA
:100F3000CF0B9B01AC0160E070E086E993E40E9476
:100F40009B0D4B015C0181E10E945D019C01990FA9
:100F5000440B550B2115F4E03F074105510524F0E2
:100F60002FEF33E040E050E057FF03C020E030E0D7
:100F7000A901A8EEB3E00E94190B2FEF33E040E087
:100F800050E00E94FA0ACA01B9010E94790C20E0DF
:100F900030E04AE754E40E94CF0B6B017C012AE069
:100FA00037ED43E25CE3C501B4010E942E0D9B01C5
:100FB000AC01C701B6010E945E0B6B017C0120E011
:100FC00030E0A9010E94CA0B87FD57C2C986DA86A4
:100FD000EB86FC8620E030E040E251E469857A85CA
:100FE0008B859C850E94290D181644F480E090E0C2
:100FF000A0E2B1E489879A87AB87BC870E946F0122
:101000006B017C018091430790914407A0914507B3
:10101000B0914607A7019601281B390B4A0B5B0BC1
:10102000CA01B9010E94770C20E034E244E759E498
:101030000E94CF0B2B013C0120E030E0A9010E946F
:10104000CA0B181644F03FE6432E32E1532E33E824
:10105000632E3AE3732EC0924307D0924407E09286
:101060004507F09246078FE00E945D01BC01990F91
:10107000880B990B0E94790C20E030EC4FE754E488
:101080000E94CF0B6D837E838F839887C984DA8417
:10109000EB84FC8426E636E646E65FE3C701B6014C
:1010A0000E942E0D4B015C012DEC3CEC4CE85FE303
:1010B000C701B6010E942E0D6D877E878F87988BA2
:1010C00045E050E04C0F5D1F5A8349833C822B82E0
:1010D00066E377E0CE0101960E94FC0469E277E0C6
:1010E000CE0101960E94FC046CE177E0CE010196EE
:1010F0000E94FC0480913607882371F02091370705
:10110000309138074091390750913A07C501B40131
:101110000E942E0D4B015C0180912907882371F0FC
:1011200020912A0730912B0740912C0750912D07D1
:10113000C701B6010E942E0D6B017C0180911C0736
:10114000882391F020911D0730911E0740911F07C1
:10115000509120076D857E858F8598890E942E0D80
:101160006D877E878F87988B20E030E040E853E4DE
:10117000C501B4010E942E0DA30192010E942E0D03
:10118000209118073091190740911A0750911B07B9
:101190000E945E0B4B015C01809218079092190728
:1011A000A0921A07B0921B0720E030E040E853E419
:1011B000C701B6010E942E0DA30192010E942E0DBF
:1011C0002091140730911507409116075091170789
:1011D0000E945E0B6B017C01C0921407D092150730
:1011E000E0921607F092170720E030E040E853E461
:1011F0006D857E858F8598890E942E0DA3019201B1
:101200000E942E0D20911007309111074091120776
:10121000509113070E945E0B2B013C014092100776
:1012200050921107609212077092130720E030E08D
:1012300040E853E4C501B4010E94290D87FD10C0A8
:1012400020E030E040E853E4C501B4010E945D0BAA
:10125000609318077093190780931A0790931B07E0
:1012600020E030E040E853E4C701B6010E94290DB8
:1012700087FD10C020E030E040E853E4C701B6012C
:101280000E945D0B609314077093150780931607F7
:101290009093170720E030E040E853E4C301B20127
:1012A0000E94290D87FD10C020E030E040E853E4A3
:1012B000C301B2010E945D0B609310077093110788
:1012C00080931207909313074091180750911907C4
:1012D00060911A0770911B0780E195E00E94A001C0
:1012E0005C014091140750911507609116077091A9
:1012F000170780E193E00E94A0016C014091100764
:1013000050911107609112077091130780E191E0ED
:101310000E94A0017C01B50160587F4F672F77279D
:10132000072E000C880B990B0E94790C2DEC3CECDD
:101330004CEC5DE30E942E0D4B015C0126E636E687
:1013400046E65FE3609108017091090180910A010E
:1013500090910B010E942E0D9B01AC01C501B401BF
:101360000E945E0B4B015C01809208019092090182
:10137000A0920A01B0920B01B60160587F4F672F0F
:101380007727072E000C880B990B0E94790C2DEC07
:101390003CEC4CEC5DE30E942E0D2B013C0126E65B
:1013A00036E646E65FE360910401709105018091A5
:1013B0000601909107010E942E0D9B01AC01C30113
:1013C000B2010E945E0B2B013C014092040150923D
:1013D00005016092060170920701B70160587F4FC6
:1013E000672F7727072E000C880B990B0E94790C2A
:1013F0002DEC3CEC4CEC5DE30E942E0D6B017C016E
:1014000026E636E646E65FE3609100017091010151
:1014100080910201909103010E942E0D9B01AC016D
:10142000C701B6010E945E0B6B017C01C0920001F6
:10143000D0920101E0920201F0920301C501B401D2
:101440000E94480C70E07093890060938800C3018B
:10145000B2010E94480C70E070938B0060938A0088
:10146000C701B6010E94480C6093B3000115110535
:1014700009F4CFCC0E940000CACC19861A861B86BC
:101480001C86A8CDECE4F7E082E390E0A0E0B0E0B9
:1014900080839183A283B38314821582168217827C
:1014A00081E0808781871286138608958F929F92AC
:1014B000AF92BF92CF92DF92EF92FF92CF93DF93E2
:1014C000EC01688179818A819B81611571058105B3
:1014D000910521F464E279ED8BE597E02DE133EF9E
:1014E00041E050E00E94FA0A49015A019B01AC0117
:1014F000A7EAB1E40E94190B6B017C01ACEEB4EFDA
:10150000A50194010E94270BC60ED71EE81EF91EE6
:10151000F7FE06C081E0C81AD108E10880E8F80AA1
:10152000C882D982EA82FB82C701B6019F77DF9128
:10153000CF91FF90EF90DF90CF90BF90AF909F90B2
:101540008F9008958F929F92AF92BF92CF92DF9229
:10155000EF92FF9260910C0170910D0180910E014C
:1015600090910F01611571058105910521F464E2E7
:1015700079ED8BE597E02DE133EF41E050E00E94FB
:10158000FA0A49015A019B01AC01A7EAB1E40E94A1
:10159000190B6B017C01ACEEB4EFA50194010E9424
:1015A000270BC60ED71EE81EF91EF7FE06C081E007
:1015B000C81AD108E10880E8F80AC0920C01D0925C
:1015C0000D01E0920E01F0920F01C701B6019F7765
:1015D000FF90EF90DF90CF90BF90AF909F908F9053
:1015E000089560930C0170930D0180930E01909308
:1015F0000F010895052E97FB1EF400940E94110B15
:1016000057FD07D00E942C0B07FC03D04EF40C941E
:10161000110B50954095309521953F4F4F4F5F4F9F
:10162000089590958095709561957F4F8F4F9F4F4E
:1016300008950E944E0BA59F900DB49F900DA49FFE
:10164000800D911D11240895B7FF0C94190B0E9471
:10165000190B821B930B0895A1E21A2EAA1BBB1B28
:10166000FD010DC0AA1FBB1FEE1FFF1FA217B3076E
:10167000E407F50720F0A21BB30BE40BF50B661F84
:10168000771F881F991F1A9469F760957095809548
:1016900090959B01AC01BD01CF010895A29FB001BF
:1016A000B39FC001A39F700D811D1124911DB29F96
:1016B000700D811D1124911D08955058BB27AA2734
:1016C0000E94750B0C94EF0C0E94E10C38F00E9404
:1016D000E80C20F039F49F3F19F426F40C94DE0C4A
:1016E0000EF4E095E7FB0C94D80CE92F0E94000D56
:1016F00058F3BA17620773078407950720F079F447
:10170000A6F50C94220D0EF4E0950B2EBA2FA02D09
:101710000B01B90190010C01CA01A0011124FF279E
:10172000591B99F0593F50F4503E68F11A16F04099
:10173000A22F232F342F4427585FF3CF4695379598
:101740002795A795F0405395C9F77EF41F16BA0B5D
:10175000620B730B840BBAF09150A1F0FF0FBB1F0B
:10176000661F771F881FC2F70EC0BA0F621F731F54
:10177000841F48F4879577956795B795F7959E3FB1
:1017800008F0B0CF9395880F08F09927EE0F979542
:10179000879508950E94B40C08F481E008950E9492
:1017A000E30B0C94EF0C0E94E80C58F00E94E10C43
:1017B00040F029F45F3F29F00C94D80C51110C949F
:1017C000230D0C94DE0C0E94000D68F39923B1F3F5
:1017D000552391F3951B550BBB27AA276217730757
:1017E000840738F09F5F5F4F220F331F441FAA1FEB
:1017F000A9F335D00E2E3AF0E0E832D091505040A7
:10180000E695001CCAF72BD0FE2F29D0660F771F54
:10181000881FBB1F261737074807AB07B0E809F03A
:10182000BB0B802DBF01FF2793585F4F3AF09E3FBF
:10183000510578F00C94D80C0C94230D5F3FE4F321
:10184000983ED4F3869577956795B795F7959F5F02
:10185000C9F7880F911D9695879597F90895E1E04E
:10186000660F771F881FBB1F621773078407BA07AD
:1018700020F0621B730B840BBA0BEE1F88F7E09508
:1018800008950E94480C6894B1110C94230D08959A
:101890000E94080D88F09F5798F0B92F9927B751EB
:1018A000B0F0E1F0660F771F881F991F1AF0BA9504
:1018B000C9F714C0B13091F00E94220DB1E0089533
:1018C0000C94220D672F782F8827B85F39F0B93F25
:1018D000CCF3869577956795B395D9F73EF49095B7
:1018E0008095709561957F4F8F4F9F4F0895E89435
:1018F00009C097FB3EF490958095709561957F4F58
:101900008F4F9F4F9923A9F0F92F96E9BB27939505
:10191000F695879577956795B795F111F8CFFAF415
:10192000BB0F11F460FF1BC06F5F7F4F8F4F9F4F46
:1019300016C0882311F096E911C0772321F09EE8A4
:10194000872F762F05C0662371F096E8862F70E00A
:1019500060E02AF09A95660F771F881FDAF7880FE4
:101960009695879597F90895990F0008550FAA0B3A
:10197000E0E8FEEF16161706E807F907C0F01216A2
:101980001306E407F50798F0621B730B840B950BA5
:1019900039F40A2661F0232B242B252B21F40895FA
:1019A0000A2609F4A140A6958FEF811D811D089597
:1019B00097F99F6780E870E060E008959FEF80EC02
:1019C000089500240A9416161706180609060895A5
:1019D00000240A9412161306140605060895092E0B
:1019E0000394000C11F4882352F0BB0F40F4BF2B7A
:1019F00011F460FF04C06F5F7F4F8F4F9F4F0895BA
:101A000057FD9058440F551F59F05F3F71F04795AF
:101A1000880F97FB991F61F09F3F79F08795089594
:101A2000121613061406551FF2CF4695F1DF08C0B3
:101A3000161617061806991FF1CF869571056105D0
:101A400008940895E894BB2766277727CB0197F978
:101A500008950E94B40C08F48FEF08950E94410D80
:101A60000C94EF0C0E94E10C38F00E94E80C20F07E
:101A7000952311F00C94D80C0C94DE0C11240C94CA
:101A8000230D0E94000D70F3959FC1F3950F50E058
:101A9000551F629FF001729FBB27F00DB11D639F20
:101AA000AA27F00DB11DAA1F649F6627B00DA11DC6
:101AB000661F829F2227B00DA11D621F739FB00D6C
:101AC000A11D621F839FA00D611D221F749F3327DC
:101AD000A00D611D231F849F600D211D822F762F75
:101AE0006A2F11249F5750409AF0F1F088234AF052
:101AF000EE0FFF1FBB1F661F771F881F91505040BE
:101B0000A9F79E3F510580F00C94D80C0C94230D3E
:101B10005F3FE4F3983ED4F3869577956795B79544
:101B2000F795E7959F5FC1F7FE2B880F911D96955E
:101B3000879597F90895FA01EE0FFF1F309621055A
:101B40003105A1F16115710561F48038BFE39B0790
:101B500049F168949038810561F08038BFEF9B07A8
:101B600041F099234AF5FF3FE1053105210519F1BF
:101B7000E8940894E795D901AA2329F4AB2FBE2F46
:101B8000F85FD0F310C0FF5F70F4A695E0F7F73967
:101B900050F019F0FF3A38F49F779F930DD00F90D3
:101BA00007FC9058089546F00C94DE0C60E070E05D
:101BB00080E89FE308954FE79F775F934F933F93AC
:101BC0002F930E94960E2F913F914F915F910E940B
:101BD0002E0D0C94F30D29F416F00C94D80C0C94E3
:101BE000220D0C94DE0C0E94080DA8F39638A0F785
:101BF00007F80F92E8942BE33AEA48EB5FE70E947C
:101C0000440D0F920F920F924DB75EB70F920E9444
:101C1000DE0EE8E6F0E00E94250E4F915F91EF9115
:101C2000FF91E595EE1FFF1F49F0FE57E06844273E
:101C3000EE0F441FFA95E1F74195550B0E94580E9F
:101C40000F9007FE0C944C0E0895DF93CF931F93D3
:101C50000F93FF92EF92DF927B018C01689406C094
:101C6000DA2EEF010E94410DFE01E894A591259125
:101C7000359145915591A6F3EF010E94750BFE0138
:101C80009701A801DA9469F7DF90EF90FF900F9128
:101C90001F91CF91DF9108959B01AC0160E070E04E
:101CA00080E89FE30C94CF0B0C94D80C0C94120F8B
:101CB0000E94080DD8F39923C9F3940F511DA3F383
:101CC0009150504094F059F0882332F0660F771FFE
:101CD000881F91505040C1F79E3F51052CF7880F47
:101CE000911D9695879597F908955F3FACF0983EC2
:101CF0009CF0BB27869577956795B79508F4B160FA
:101D00009395C1F7BB0F58F711F460FFE8CF6F5FF1
:101D10007F4F8F4F9F4FE3CF0C94230D16F00C9401
:101D2000120F0C94DE0C68940C94D80C0E94080DD1
:101D3000A8F39923C1F3AEF3DF93CF931F930F93CF
:101D4000FF92C92FDD2788232AF02197660F771F7E
:101D5000881FDAF720E030E040E85FEB9FE3883946
:101D600020F0803E38F021968F770E945E0BE0E9EC
:101D7000F0E004C00E945E0BEDEBF0E00E94250E47
:101D80008B01BE01EC01FB2E6F5771097595771F12
:101D9000880B990B0E94790C28E132E741E35FE35D
:101DA0000E94410DAF2D9801AE01FF900F911F9140
:101DB000CF91DF910E94750B0C94EF0CFA01DC01BE
:101DC000AA0FBB1F9B01AC01BF5728F42227332762
:101DD0004427507820C0B75190F4AB2F002446958B
:101DE00037952795011CA395D2F3002071F0220F9F
:101DF000331F441FB395DAF30ED00C945D0B6130A2
:101E00007105A0E88A07B94630F49B01AC0166274A
:101E1000772788279078309621F02083318342837A
:101E2000538308959F3F31F0915020F48795779523
:101E30006795B795880F911D9695879597F90895A1
:101E4000EE0FFF1F0590F491E02D0994F894FFCF59
:101E500000000043000000430000004301000000B8
:00000001FF
